:020000040800F2
:1000000000040020E1010008E3010008E30100080A
:10001000E3010008E3010008E3010008E301000830
:10002000E3010008E3010008E3010008D52D000802
:10003000E3010008E3010008E3010008E301000810
:10004000E3010008E3010008E3010008E301000800
:10005000E3010008E30100083930000865300008BA
:1000600091300008BD300008E9300008E3010008C5
:10007000E3010008E3010008E3010008E3010008D0
:10008000E3010008E3010008E3010008E3010008C0
:10009000E3010008E3010008E3010008153100084E
:1000A000E3010008E3010008E3010008E3010008A0
:1000B000E3010008E3010008E3010008E301000890
:1000C000E3010008E3010008E3010008E301000880
:1000D000E3010008E3010008E3010008E301000870
:1000E0007D310008E3010008E3010008E301000896
:1000F000E3010008E3010008E3010008E301000850
:10010000E3010008E3010008512E0008E3010008A4
:10011000E3010008E3010008E3010008E30100082F
:10012000E3010008E3010008E3010008E30100081F
:10013000E3010008E3010008E3010008E30100080F
:10014000E3010008E3010008E30100081D250008A1
:10015000E3010008E3010008E3010008E3010008EF
:10016000E3010008E3010008E3010008E3010008DF
:10017000E3010008E3010008E3010008E3010008CF
:10018000E3010008E3010008E3010008E3010008BF
:10019000E3010008E3010008E3010008E3010008AF
:1001A000E3010008E3010008E3010008E30100089F
:1001B000E3010008E3010008E3010008E30100088F
:1001C000E3010008E3010008E3010008E30100087F
:1001D000E3010008E3010008E3010008E30100086F
:1001E00002E000F000F8FEE772B6394880F30888B4
:1001F000384880F3098838484EF60851CEF200019D
:10020000086040F20000CCF200004EF63471CEF2ED
:1002100000010860BFF34F8FBFF36F8F40F2000003
:10022000C0F2F0004EF68851CEF200010860BFF334
:100230004F8FBFF36F8F4FF00000E1EE100A4EF6C4
:100240003C71CEF200010860062080F31488BFF3F1
:100250006F8F01F02BFE02F053FD4FF055301F4918
:100260001B4A91423CBF41F8040BFAE71C49194A6A
:1002700091423CBF41F8040BFAE71A491A4A1B4B5A
:100280009A423EBF51F8040B42F8040BF8E70020F5
:100290001749184A91423CBF41F8040BFAE701F0B4
:1002A00009FE02F089FD144C144DAC4203DA54F8F7
:1002B000041B8847F9E700F03FF8114C114DAC42A0
:1002C00003DA54F8041B8847F9E701F0F1BD000098
:1002D000000400200024002000000008000000208E
:1002E00000040020B035000800240020282400204D
:1002F0002824002018340020E0010008E001000854
:10030000E0010008E00100082DE9F04F2DED108A12
:10031000C1F80CD0C3689D46BDEC108ABDE8F08FD3
:10032000002383F311882846A047002001F080FABB
:1003300001F030FA00DFFEE71A4B472270B51A7061
:10034000052200245A700F229C70DC701C715C71B5
:100350009C71DC711C725C729A72DC7201F074FD2B
:10036000064601F09DFD054650B90F4B9E4217D041
:1003700001339E4241F2883412BF05460024012514
:10038000002001F067FD0DB100F0B4F800F0F6FCBC
:1003900000F0C0FB204600F00BF900F0ABF8F9E7E5
:1003A0000446EDE728240020010007B008B500F05E
:1003B00053FBA0F120035842584108BD07B5054B37
:1003C00002211B88ADF8043001A800F093FB03B0B4
:1003D0005DF804FB78320008064991F8243033B107
:1003E00000230822086A81F8243000F0B5BB012000
:1003F000704700BF482400202DE9F84F234C94F8A3
:1004000024300546884617468BBB2E46DFF87C9085
:10041000002F38D094F824A0BAF1000F05D1202283
:10042000FF214846266200F097FCCAF10805BD424C
:1004300028BF3D465FFA85FBAD0041462A4604EBE6
:100440008A0000F05FFC94F82430A7EB0B079B4474
:100450005FFA8BFBBBF1080F2E44A844FFB284F86F
:1004600024B0D5D1FFF7B8FF0028D1D108E0266A23
:1004700006EB8306B042C9D0FFF7AEFF0028C4D117
:100480000020BDE8F88F0120BDE8F88F4824002047
:1004900010B5202383F311881248C3680BB101F013
:1004A0004DFA0023104A0F484FF47A7101F00AFA0E
:1004B000002383F311880D4C236813B12368013B9B
:1004C0002360636813B16368013B6360084B1B786A
:1004D00033B9636823B9022000F000FC3223636063
:1004E00010BD00BF342400209104000878290020AA
:1004F0007024002010B5254B254953F8042F0132F4
:1005000000D110BD8B42F8D1224C234B22689A4275
:100510003AD9224B9B6803F1006303F580339A427A
:1005200032D2002000F010FB1D4B0220187000F0AA
:10053000C5FB1C4B1A6C00221A64196E1A66196EE0
:10054000596C5A64596E5A665A6E5A6942F0800262
:100550005A615A6922F080025A615A691A6942F056
:1005600000521A611A6922F000521A611B6972B6B0
:100570000D4A0E4B13601B682268202181F31188FD
:100580009D4683F30888104710BD00BFFCFF00089C
:100590001C00010804000108FFFF000828240020B7
:1005A000702400200038024008ED00E0000001083F
:1005B0002DE9F04FB54C97B020228246FF210EA8BE
:1005C000A56800F0C9FBB24A1378A046A3B9B148A8
:1005D0000121C3601170202383F31188C3680BB11C
:1005E00001F0ACF90023AC4AAA484FF47A7101F04B
:1005F00069F9002383F31188DFF8BCB2BAF1000F68
:1006000001D0CBF800A0A54F00243C70CBF80440EB
:100610002646012000F052FBBAF1000F00F0E08105
:10062000DBF80030002B40F0DB8117B0BDE8F08F25
:100630000220FFF7BBFE002840F0D081984B1B88BA
:10064000ADF82430022109A800F054FAE1E74FF494
:100650007A7000F001FA031E0193EFDB0220FFF72E
:10066000A5FE81460028E9D0019B581E0428E5D844
:10067000DFE800F0030C0F12150016A8052340F860
:10068000343D042100F036FA4C4650E004217F4806
:10069000F8E704218348F5E704218348F2E71C24A6
:1006A000204600F053FA04340990042109A800F010
:1006B00021FA2C2CF4D1E7E7002EBFD0002CBDD0BE
:1006C0000220FFF773FE064610B901242646B5E75F
:1006D000012000F039FA0220387000F0EFFA00240F
:1006E000E3B21846019300F03FFA814648B1019BFE
:1006F000184600F049FA01340028F1D134466B4B1A
:100700009DE7012302203B7000F0C6FA4D46D8F861
:1007100008309D4206D2284600F018FA0130EDD18B
:100720000435F4E700253D70CBF80450344600F062
:100730001BFBFFF743FE4EE1002E3FF47FAF002C82
:100740003FF47CAF0220387000F0B8FA322000F09D
:1007500083F9041EB9DB14F00306B6D1D8F80820DB
:100760002B199342B1D8B4F5807FAED8DFF8409111
:10077000A6420CDA4FF47A7000F06EF90390039BF6
:10078000002BA2DB039B06F809300136F0E7C820F6
:10079000FFF70CFE0646002897D01F2D11D8C5F193
:1007A0002009A14528BFA1460EAB25F003004A460B
:1007B0003F49184400F0A6FA4A46FF213C4800F0A1
:1007C000CBFA4FEAA4095FFA89F239492846FFF7C4
:1007D00013FE0446002891D005EB89050646A6E7DE
:1007E0000220FFF7E3FD00283FF428AFFFF7F4FDF8
:1007F00000283FF423AF4FF0000AD146D8F8083064
:100800009A453CD2BAF11F0F1CD80E9B013319D068
:100810002AF0030316AA134453F8203C09932549F0
:100820004B68A3B1002209A8135C83EA0903DBB279
:10083000013251F82330042A83EA1929F4D10AF14C
:10084000040ADBE7504600F081F90990E7E71A4611
:10085000082012F0010F4FEA52021FBF82F06D42D2
:1008600082F4380282F4034282F020020138F0D18F
:1008700041F823200133B3F5807FE8D1D2E716A8F1
:10088000042140F8489D00F035F950E72824002065
:1008900074250020342400209104000870240020D6
:1008A0007A3200082C240020302400207C320008FA
:1008B00074240020782500207829002016A8002321
:1008C00040F8343D642100F0F1F800287FF4B6AE22
:1008D0000220FFF76BFD00283FF4B0AE099800F04E
:1008E00065F916AB43F8440D04211846CBE716A86A
:1008F000002340F8343D642100F0D8F800287FF44C
:100900009DAE0220FFF752FD00283FF497AE0998F4
:1009100000F05AF916AB43F8400DE5E70220FFF767
:1009200045FD00283FF48AAE00F054F916AB43F8B9
:100930003C0DD9E70220FFF739FD00283FF47EAED9
:1009400009A9142000F04CF9814616A8042140F8AA
:10095000389D00F0CFF8494609A894E74FF47A7023
:10096000FFF724FD00283FF469AEFFF735FD0028AE
:100970003FF4C5AE0E9B01330CD008220EA9002017
:10098000FFF73AFD00283FF4BAAE2022FF210EA85F
:1009900000F0E2F9FFF712FD2E4800F04FFF44E6A9
:1009A00016A8002340F8343D642100F07FF80028A9
:1009B0007FF444AE0220FFF7F9FC00283FF43EAE7E
:1009C000FFF7FCFC41F2883000F038FF099800F096
:1009D000FFF900F0C9F94FF0000A1AE60646A6E64C
:1009E000002000F039F80390039B002BFFF614AEB3
:1009F000012000F051F9039B213B122B3FF609AE79
:100A000001A252F823F000BF310600084F0600088B
:100A1000B9060008130600081306000813060008AC
:100A20003907000813060008E1070008BD080008A0
:100A3000EF0800081D090008130600083509000822
:100A4000130600085D0900082F07000813060008B8
:100A5000A1090008A086010037B5114B1A780132B0
:100A6000D2B20024012A01468DF8074011D80D4862
:100A700003681D6A4FF47A734B4301220DF107019D
:100A8000A847012805D1084B9DF807001C7003B04A
:100A900030BD4FF4FA7000F0D1FE4FF0FF30F6E7B2
:100AA00000240020C82900208429002038B50E4BDE
:100AB0001A780132D2B2012A05460ED80B480368D3
:100AC0001C6A4FF47A734B4304222946A04704283A
:100AD00003D1074B0020187038BD4FF4FA7000F0B6
:100AE000ADFE4FF0FF3038BD00240020C8290020A3
:100AF0008429002030B4054C2368DD69044B0A4684
:100B0000AC460146204630BC604700BFC8290020E3
:100B1000A086010070B501F0D9F8094C094E20708B
:100B2000002530682378834208D901F0C9F833687A
:100B300005440133B5F5803F3360F2D370BD00BF8B
:100B4000852900208029002001F06AB900F10060A9
:100B500000F580300068704700F10060920000F5F9
:100B6000803001F0F5B80000054B1A68054B1B7882
:100B70009B1A834202D9104401F0A2B800207047AA
:100B8000802900208529002038B5074D04462868B3
:100B9000204401F09DF828B928682044BDE8384079
:100BA00001F0AEB838BD00BF8029002010F003036B
:100BB00008D1B0F5007F05D800F10050A0F508403D
:100BC0000068704700207047014BC058704700BF55
:100BD000107AFF1F014B1868704700BF002004E027
:100BE00070B52A4B1C68C4F30B03240C63B140F2AC
:100BF0001342934231D040F2194293422FD040F237
:100C0000214293422DD10323214A0C2505FB0323C6
:100C10005D6893F9082042F201039C4224D0B4F5A8
:100C2000805F23D041F201039C4221D041F20303B3
:100C30009C421FD041F207039C4208BF3122441E50
:100C40000C44013D0B46A3421ED215F9016F581CFE
:100C500096B1034600F8016CF5E70123D4E70223BF
:100C6000D2E73F220B4DD6E73322E3E74122E1E70B
:100C70005A22E4E75922E2E72C2584421D7001D96B
:100C8000981C5A70401A70BD1846FBE7002004E01B
:100C90008C32000880320008022804D1054B4FF046
:100CA00080429A6170470128FCD14FF40012024B38
:100CB000F7E700BF000C024000080240022804D100
:100CC000044B4FF480429A6170470128FCD12022E6
:100CD000014BF8E7000C024000080240022805D151
:100CE000064A536983F48043536170470128FCD15D
:100CF000034A536983F02003F6E700BF000C02406B
:100D00000008024010B50023934203D0CC5CC454C9
:100D10000133F9E710BD000030B5441E14F9010F8E
:100D20000B4660B193F90050854201F1010106D1F3
:100D30001AB993F90020801A30BD013AEEE7002A73
:100D4000F7D1104630BD000002460346981A13F949
:100D5000011B0029FAD1704702440346934202D096
:100D600003F8011BFAE77047024B1A78024B1A701E
:100D7000704700BF842900200024002038B5104DA2
:100D8000104C284600F0A2F82146284600F0CAF888
:100D900023680D485A6DD2F8043843F00203C2F8B4
:100DA000043800F04BFD0949206800F0C7F92368BA
:100DB0005A6DD2F8043823F00203C2F8043838BD63
:100DC000C82900205833000840420F00AC33000807
:100DD00070470000026843681143016003B118477F
:100DE0007047000013B5446BD4F894341A68117836
:100DF000042915D1217C022912D1197912890123E4
:100E00008B4013420CD101A904F14C0001F0ECFD20
:100E1000D4F89444019B21790246206800F0DAF965
:100E200002B010BD143001F06FBD00004FF0FF3371
:100E3000143001F069BD00004C3001F041BE0000EB
:100E40004FF0FF334C3001F03BBE0000143001F096
:100E50003DBD00004FF0FF31143001F037BD000000
:100E60004C3001F00DBE00004FF0FF324C3001F06D
:100E700007BE0000D0F8942438B513681978042907
:100E8000054601D0012038BD017C0229FAD1127932
:100E90005C89012090400440F4D105F1140001F078
:100EA000CFFC02460028EDD0D5F894544FF480735F
:100EB0002868697900F07CF9204638BD406BFFF75F
:100EC000D9BF000000207047704700007FB5124B6B
:100ED0000360002343608360C360012502260F4B3B
:100EE000057404460290019300F18402294600969D
:100EF0004FF48073143001F07FFC094B019302948E
:100F000000964FF4807304F52372294604F14C00D7
:100F100001F046FD04B070BDDC320008BD0E0008D3
:100F2000E50D00080B68202282F311880A7903EB93
:100F3000820290614A79093243F822008A7912B11B
:100F400003EB8203986102230374C0F89414002316
:100F500083F311887047000038B5037F044613B14E
:100F600090F85430ABB9201D01250221FFF732FF64
:100F700004F1140025776FF0010100F087FC84F87C
:100F8000545004F14C006FF00101BDE8384000F00E
:100F90007DBC38BD10B5012104460430FFF71AFFAF
:100FA0000023237784F8543010BD000038B5044680
:100FB0000025143001F038FC04F14C00257701F0D5
:100FC00007FD201D84F854500121FFF703FF204640
:100FD000BDE83840FFF74EBF90F8443003F060039F
:100FE000202B19D190F84520212A0AD0222A4FF02F
:100FF00000030ED0202A0FD1084A82630722C26361
:1010000004E0064B83630723C363002303640120CA
:1010100070478363C363F9E7002070470124002011
:10102000D0F8943437B51A681178042904461AD1D7
:10103000017C022917D11979128901238B401342AF
:1010400011D100F14C05284601F082FD58B101A9EB
:10105000284601F0C9FCD4F89444019B217902464A
:10106000206800F0B7F803B030BD000000EB81034A
:10107000F7B59C6905460E46F4B1202383F3118829
:1010800005EB8607201D0821FFF7A4FEFB685B69BE
:101090001B684C3413B1204601F0B4FC01A9204672
:1010A00001F0A2FC024648B1019B3146284600F0FF
:1010B00091F8002383F3118803B0F0BDFB685A69EF
:1010C0001268002AF5D01B8A013B1340F1D105F1CB
:1010D0004402EAE7093138B550F82140DCB1202359
:1010E00083F31188D4F894241368527903EB8203B4
:1010F000DB689B695D6845B104216018FFF76AFEF3
:10110000294604F1140001F0A5FB2046FFF7B2FECA
:10111000002383F3118838BD7047000000F050BFF2
:101120000123037000234360C36183620362C362CF
:1011300043620363038143817047000038B504466E
:10114000202383F3118800254160C5600561456156
:10115000856100F045FF0223237085F3118838BDB7
:1011600070B500EB810305465069DA600E461446FF
:1011700018B110220021FFF7EFFDA06918B110226D
:101180000021FFF7E9FD31462846BDE8704000F038
:10119000F1BF0000028902F001020281428902F0DF
:1011A00001024281002202614261826101F076B84F
:1011B000F0B400EB81044789E4680125A4698D40FF
:1011C0003D43458123600023A2606360F0BC01F0D1
:1011D00091B80000F0B400EB81040789E4680125B0
:1011E00064698D403D43058123600023A2606360F4
:1011F000F0BC01F00BB9000070B5022300250446D5
:101200000370A0F84C5080F84E5080F84F50058184
:101210004581C56005614561856180F8345000F005
:1012200045FF63681B6823B129462046BDE870402E
:10123000184770BD436802781B6880F8502005226B
:1012400002700BB10421184770470000436890F802
:1012500050201B6802700BB1052118477047000031
:1012600090F8343070B5044613B1002380F8343060
:1012700004F14402204601F033F863689B6863BBC5
:1012800094F8445015F0600615D194F8453005F0F7
:101290007F0545EA032540F202339D4200F00E81AE
:1012A0005BD8022D00F0DC803FD8002D00F0878055
:1012B000012D00F0CF800021204601F069FA0021C5
:1012C000204601F05BFA63681B6813B106212046D3
:1012D0009847062384F8343070BD2046984700288C
:1012E000CED094F84B2094F84A3043EA0223E26BC4
:1012F000934238BFE36394F94430E56B002B4FF021
:10130000200380F2FD80002D00F0EC80092284F89B
:10131000342083F311880021E36BA26B2046FFF792
:1013200059FF002383F3118870BDB5F5817F00F06C
:10133000B180B5F5407F49D0B5F5807FBBD194F839
:101340004630012BB7D1B4F84C3023F00203A4F897
:101350004C30A663E6632664C3E740F201639D4216
:101360001ED8B5F5C06F3BD2B5F5A06FA3D1B4F8C8
:101370004430B3F5A06F0ED194F8463084F84E3067
:10138000204600F0EBFE63681B6813B10121204684
:101390009847032323700023A363E3632364A0E738
:1013A000B5F5106F32D040F602439D4252D0B5F5EC
:1013B000006F80D104F14F03A363012324E004F103
:1013C0004C03A3630223E36325648AE794F8463061
:1013D000012B7FF470AFB4F84C3043F00203B6E752
:1013E00094F84920616894F848304D6894F84710A3
:1013F00043EA0223204694F84620A84700283FF4F9
:101400005AAF4368A3630368E363A4E72378042B1C
:1014100010D1202383F311882046FFF7BBFE86F30B
:101420001188636884F84F601B68032121700BB139
:101430002046984794F84630002BACD084F84F30C3
:101440000423237063681B68002BA4D0022120466C
:101450009847A0E7374BA3630223E36300239DE78C
:1014600094F8481011F0800F204601F00F010ED0C3
:1014700000F028FF012806D002287FF41CAF2E4B75
:10148000A363E06367E72D4BA363E56363E700F0C5
:101490000BFFEFE794F84630002B7FF40CAF94F885
:1014A000483013F00F013FF476AF1A06204602D5FC
:1014B00001F082F96FE701F075F96CE794F84630B6
:1014C000002B7FF4F8AE94F8483013F00F013FF48E
:1014D00062AF1B06204602D501F05AF95BE701F026
:1014E0004DF958E7142284F8342083F311882B46F1
:1014F0002A4629462046FFF75BFE85F3118870BD1A
:101500005DB1152284F8342083F311880021E36B48
:10151000A26B2046FFF74CFE03E70B2284F8342031
:1015200083F311882B462A4629462046FFF752FEB0
:10153000E3E700BF0C330008043300080833000859
:1015400038B590F834300446152B29D8DFE803F07D
:101550003E28282828283E28280B293928282828EA
:10156000282828283E3E90F84B1090F84A20C36B5C
:1015700042EA01229A4214D9C268128AB3FBF2F5F8
:1015800002FB15356DB9202383F311882B462A46BB
:101590002946FFF71FFE85F311880A2384F83430AB
:1015A00038BD142384F83430202383F311880023BA
:1015B0001A4619462046FFF7FBFD002383F31188E6
:1015C00038BD036C03B198470023E7E7002101F021
:1015D000DFF80021204601F0D1F863681B6813B1E1
:1015E0000621204698470623D8E7000090F83420CB
:1015F000152A38B5044622D80123934040F64162AB
:1016000013421DD113F480150FD19B0217D50B2364
:1016100080F83430202383F311882B462A4629464C
:10162000FFF7D8FD85F3118838BDC3689B695B68F7
:101630002BB9036C03B19847002384F8343038BDCC
:10164000002101F0A5F80021204601F097F8636819
:101650001B6813B10621204698470623EDE70000DA
:10166000024B00221B605B609A6070478829002053
:10167000002303748268054B1B6899689142FBD272
:101680005A680360426010605860704788290020E3
:1016900008B5202383F31188037C032B05D0042B8A
:1016A0000DD02BB983F3118808BD436900221A605D
:1016B0004FF0FF334361FFF7DBFF0023F2E790E8D1
:1016C0000C001A6002685360F2E700000023037404
:1016D0008268054B1B6899689142FBD85A68036081
:1016E000426010605860704788290020054B1969D6
:1016F0000874186802681A60536018610123037443
:10170000FEF702BE8829002030B54B1C87B0054685
:101710000A4C10D023690A4A01A800F0D3F82846E1
:10172000FFF7E4FF049B13B101A800F007F9236958
:10173000586907B030BDFFF7D9FFF8E788290020C6
:101740009116000838B50C4D41612B6981689A6883
:101750009142044603D8BDE83840FFF789BF1846D8
:10176000FFF786FF01232C61014623742046BDE864
:101770003840FEF7C9BD00BF88290020044B1A6815
:101780001B6990689B68984294BF002001207047B5
:101790008829002010B5084C236820691A68226047
:1017A0005460012223611A74FFF790FF01462069FB
:1017B000BDE81040FEF7A8BD882900208260022203
:1017C00002740022427470478368A3F17C0243F8DC
:1017D0000C2C026943F83C2C426943F8382C074A28
:1017E00043F81C2CC26843F8102C022203F8082C82
:1017F000002203F8072CA3F118007047210300080A
:1018000010B5202383F31188FFF7DEFF0021044683
:10181000FFF798FF002383F31188204610BD0000D6
:10182000024B1B6958610F20FFF760BF8829002019
:10183000202383F31188FFF7F3BF000008B50146AA
:10184000202383F311880820FFF75EFF002383F332
:10185000118808BD49B1064B42681B6918605A607F
:10186000136043600420FFF74FBF4FF0FF30704715
:10187000882900200368984206D01A6802605060E8
:1018800059611846FFF7F4BE7047000038B50446AA
:101890000D462068844200D138BD036823605C6037
:1018A0004561FFF7E5FEF4E7054B03F114025A61C9
:1018B0009A614FF0FF32DA6100221A62704700BF6E
:1018C00088290020F8B503611A4BC2605C6A1A4B84
:1018D0001A46022952F8145F38BF02219542064683
:1018E0001F460AD1586198611C620560456081609D
:1018F0000819BDE8F84001F04DB9186AAB68241A20
:101900000C1902D3E41A2D6804E09C4202D2204450
:1019100001F050F9AB689C42F4D86B687360356095
:101920001E606E60B460A9684FF0FF33091BA960A8
:10193000FB61F8BD000C00408829002010B41A4C4F
:10194000234653F8141F814210D0416802680A6090
:10195000026851609A424FF00001C16003D0936861
:1019600081680B4493605DF8044B70470A686261BC
:1019700000209A425360C86003D15DF8044B01F027
:1019800013B99368886803449360084A206A526ACE
:10199000121A9342E7D9991A012998BF931C184447
:1019A0005DF8044B01F006B988290020000C0040C6
:1019B00000207047FEE70000704700004FF0FF3046
:1019C00070470000022906D0032906D001290648E5
:1019D00018BF0020704705487047032A9ABF044883
:1019E00000EBC2000020704708340008BC33000838
:1019F0000824002070B5044608460D46FFF7A4F9F8
:101A0000C6B22046013403780BB9184670BD324681
:101A10002946FFF781F90028F3D1012070BD0000AD
:101A20002DE9F04F81469BB008460C461646FFF75D
:101A30008BF93C49C5B22046FFF7DCFF08B10535FC
:101A4000EDB239492046FFF7D5FF08B11035EDB2A8
:101A5000632D01AF0CD8DFF8DCA0DFF8DCB03D4629
:101A600094F80080B8F1000F1CD185F8008003E0E5
:101A70002146384601F0F8FB3846FFF765F9C0B259
:101A8000431C5B0089E84800337003237370002314
:101A900002361946DAB2904206F102063AD81BB075
:101AA000BDE8F08FB8F1250F2FD107221D49204640
:101AB000FFF732F958B9DBF800202A60DBF8042080
:101AC0006A60DBF80820AA6007340C35C8E70822F2
:101AD00015492046FFF720F9B8B91448AA1C10F898
:101AE000011F134B4FEA111E01F00F011EF80AE00F
:101AF00011F80A1002F802EC984202F8011C02F1F7
:101B00000202ECD118350834AAE785F800800134C8
:101B10000135A5E7FA5C06F8022C06F8011C013332
:101B2000B8E700BF60330008683300080F7AFF1F72
:101B30001B7AFF1F7E3300087133000808B520238D
:101B400083F311880348FFF76BFA002383F31188AE
:101B500008BD00BFC829002010B50446052916D8C5
:101B6000DFE801F016150316161D202383F31188F4
:101B70000E4A0121FFF7F4FA20460D4A0221FFF731
:101B8000EFFA0C48FFF712FA002383F3118810BD17
:101B9000202383F311880748FFF7DEF9F4E72023B9
:101BA00083F311880348FFF7F5F9EDE710330008D8
:101BB00034330008C829002038B50C4D0C4C0D49B1
:101BC0002A4604F10800FFF72BFF05F1CA0204F1D1
:101BD00010000949FFF724FF05F5CA7204F1180047
:101BE0000649BDE83840FFF71BBF00BF902E00201C
:101BF0000824002090330008A1330008683300084F
:101C0000BFF34F8F024AD368DB03FCD4704700BF99
:101C1000003C024008B5094B1B7873B9FFF7F0FF91
:101C2000074B1A69002ABFBF064A5A6002F1883280
:101C30005A601A6822F480621A6008BDEE300020F3
:101C4000003C02402301674508B50B4B1B7893B954
:101C5000FFF7D6FF094B1A6942F000421A611A6871
:101C600042F480521A601A6822F480521A601A688C
:101C700042F480621A6008BDEE300020003C024051
:101C80000B2870B513D80B4A0B4C137863B90B4E65
:101C90004FF0006144F8231056F8235001330C2B09
:101CA0002944F7D10123137054F8200070BD00209F
:101CB00070BD00BF20310020F03000202834000823
:101CC000014B53F820007047283400080C2070475F
:101CD0000B2810B5044601D9002010BDFFF7D0FF36
:101CE000064B53F824301844C21A0BB9012010BD1A
:101CF00012680132F0D1043BF6E700BF2834000837
:101D00000B2810B504461ED8FFF77AFFFFF782FFB5
:101D10000E49F323CB60FFF773FFC300DBB243F43C
:101D2000007343F002030B610B6943F480330B61D2
:101D3000FFF766FFFFF7A4FFFFF786FF2046BDE829
:101D40001040FFF7C5BF002010BD00BF003C02409F
:101D50002DE9F84312F00103154643D10244B2F1D4
:101D6000016F3FD22C4B1B6813F001033AD02B4C70
:101D7000FFF750FFF323E360FFF742FF40F2012734
:101D8000032D16D8254C0F46401A40F20118EB1BC4
:101D90000B44012B00EB0706236926D823F001032F
:101DA0002361FFF751FF0120BDE8F883043D0430B3
:101DB000E6E78307E6D1236923F4407323612369AF
:101DC0003B43236151F8046B0660BFF34F8FFFF76D
:101DD00017FF03689E42E9D0236923F001032361C2
:101DE000FFF732FF0020BDE8F88323F4407323613E
:101DF000236943EA08032361B94637F8023B33807D
:101E0000BFF34F8FFFF7FCFE3688B9F80030B6B24B
:101E1000B342BCD0E0E700BF00380240003C0240C3
:101E2000084908B50B7828B153B9FFF7F3FE012331
:101E30000B7008BD23B1BDE808400870FFF704BF70
:101E400008BD00BFEE300020014B186D704700BF89
:101E500000280040094B1A6F120407D41A6F42F48D
:101E600000721A671A6F42F400421A67044A136834
:101E700043F480731360034B1865704700380240C9
:101E80000070004000280040034B1B689B0042BFCD
:101E9000024B01221A707047743802402131002031
:101EA000014B1878704700BF2131002070470000B7
:101EB000FEE70000084A094B09498B4204D3094A4E
:101EC0000021934205D3704752F8040F43F8040BE6
:101ED000F3E743F8041BF4E7D43500081834002076
:101EE0001834002018340020836D30B500229D681E
:101EF000446D11464FF0FF3004EB4213013295421E
:101F0000C3F80019C3F81019C3F80809C3F8001B77
:101F1000C3F8101BC3F8080BEED24FF00113C4F83E
:101F20001C3830BD890141F02001016103699B0625
:101F3000FCD4122000F0CABE204B03EB80022DE936
:101F4000F047D2F80CE05D6DDEF81420461CD2F8A4
:101F500000C005EB063605EB4018516861450BD310
:101F6000D5F83428012303FA00F022EA0000C5F86E
:101F700034081846BDE8F087BEF81040ACEB01030A
:101F8000A34228BF2346D8F81849A4B2B3EB840F64
:101F900010D894681F46A4F1040959F804AFC6F894
:101FA00000A0042F01D9043FF7E71C440B449460C0
:101FB0005360D2E70020BDE8F08700BF2431002045
:101FC00010B5054C2046FFF7ABF84FF0A043636512
:101FD000024BA36510BD00BF243100207C340008F3
:101FE0000378012B70B5054650D12A4B446D9842B9
:101FF0001BD1294B5A6B42F080025A635A6D42F052
:1020000080025A655A6D5A6942F080025A615A69D3
:1020100022F080025A610E2143205B6900F0D6FB5A
:102020001E4BE3601E4BC4F800380023C4F8003E8A
:10203000C02323606E6D4FF40413A3633369002B38
:10204000FCDA012333610C2000F040FE3369DB072A
:10205000FCD4122000F03AFE3369002BFCDA002693
:10206000A6602846FFF740FF6B68C4F81068DB687D
:10207000C4F81468C4F81C684BB90A4BA3614FF04C
:10208000FF336361A36843F00103A36070BD064B97
:10209000F4E700BF24310020003802404014004023
:1020A00003002002003C30C0083C30C0F8B5446D4D
:1020B000054600212046FFF735FFA96D00234FF0AC
:1020C00001128F68C4F834384FF00066C4F81C2839
:1020D0004FF0FF3004EB431201339F42C2F8006916
:1020E000C2F8006BC2F80809C2F8080BF2D20B68FC
:1020F0006A6DEB65636210231361166916F01006B2
:10210000FBD1122000F0E2FDD4F8003823F4FE6386
:10211000C4F80038A36943F4402343F01003A361DB
:102120000923C4F81038C4F814380A4BEB604FF098
:10213000C043C4F8103B084BC4F8003BC4F8106916
:10214000C4F80039EB6D03F1100243F48013EA6523
:10215000A362F8BD5834000840800010426D90F82A
:102160004E10D2F8003823F4FE6343EA0113C2F89C
:10217000003870472DE9F0410EB200EB86080D469D
:10218000D8F80C100F6807F00303022B50D0032B74
:1021900050D03D4A3D4F012B18BF1746446D4FEAC2
:1021A000451E04EB0E030022C3F8102B8A6905F1CB
:1021B000100C002A40D04A8A05F158035B013A43CB
:1021C000E2500123D4F81C2803FA0CF31343A6446D
:1021D0004A69C4F81C380023CEF8103905F13F03D2
:1021E000002A39D00A8A898B9208012988BF4A437C
:1021F000C16D04EB8303561841EA0242C6652946C5
:102200005A602046FFF78EFED8F80C301B8A43EA4E
:1022100085531F4305F148035B01E7500123D4F8C0
:102220001C2803FA05F51543C4F81C58BDE8F081D5
:10223000174FB3E7174FB1E704EB4613D3F8002B62
:1022400022F40042C3F8002BD4F81C28012303FA1F
:102250000CF322EA0303BAE704EB83030E4A5A6045
:1022600004EB461629462046FFF75CFED6F80039F7
:1022700023F40043C6F80039D4F81C38012202FACE
:1022800005F523EA0505CFE7008000100080041063
:102290000080081000800C1000040002826D12689B
:1022A000C265FFF721BE00005831436D49015B58FC
:1022B00013F4004004D013F4001F14BF01200220C7
:1022C000704700004831436D49015B5813F40040EA
:1022D00004D013F4001F14BF012002207047000037
:1022E00000EB8101CB68196A0B6813604B6853607F
:1022F0007047000000EB810330B5DD68AA69136800
:10230000D36019B9402B84BF402313606B8A1468D3
:10231000426D1C44013CB4FBF3F46343033323F0EC
:10232000030302EB411043EAC44343F0C043C0F847
:10233000103B2B6803F00303012B09B20ED1D2F836
:10234000083802EB411013F4807FD0F8003B14BF33
:1023500043F0805343F00053C0F8003B02EB4112BE
:10236000D2F8003B43F00443C2F8003B30BD00000C
:102370002DE9F041244D6E6D06EB40130446D3F871
:10238000087BC3F8087B38070AD5D6F81438190734
:1023900006D505EB84032146DB6828465B68984731
:1023A000FA072FD5D6F81438DB072BD505EB8403B5
:1023B000D968CCB98B69488A5E68B6FBF0F200FB3D
:1023C00012628AB91868DA6890420DD2121A83E84C
:1023D0001400202383F311880B482146FFF78AFF5E
:1023E00084F31188BDE8F081012303FA04F26B89BC
:1023F00023EA02036B81CB6823B121460248BDE882
:10240000F0411847BDE8F0812431002000EB810342
:1024100070B5DD68436D6C692668E6604A0156BB9D
:102420001A444FF40020C2F810092A6802F003028F
:10243000012A0AB20ED1D3F8080803EB421410F4B3
:10244000807FD4F8000914BF40F0805040F0005065
:10245000C4F8000903EB4212D2F8000940F004402E
:10246000C2F80009D3F83408012202FA01F101434D
:10247000C3F8341870BD19B9402E84BF40202060C5
:1024800020682E8A841940F00050013C1A44B4FBA5
:10249000F6F440EAC440C6E7F8B504461E48456D68
:1024A00005EB4413D3F80869C3F80869F10717D599
:1024B000D5F81038DA0713D500EB8403D9684B69D7
:1024C0001F68DA68974218D2D21B00271A605F6033
:1024D000202383F311882146FFF798FF87F31188A3
:1024E000330617D5D5F834280123A340134211D061
:1024F0002046BDE8F840FFF71FBD012303FA04F2B0
:10250000038923EA020303818B68002BE8D021466C
:102510009847E5E7F8BD00BF2431002096482DE933
:10252000F84F456D6E69AB691E4016F4805F6E61B1
:10253000044605D0FEF760FEBDE8F84F00F05ABC37
:10254000002E12DAD5F8003E8B489B071EBFD5F847
:10255000003E23F00303C5F8003ED5F8043823F00D
:102560000103C5F80438FEF771FE370502D582482D
:10257000FEF760FEB0040CD5D5F8083813F0060F4E
:10258000EB6823F470530CBF43F4105343F4A0538F
:10259000EB60310704D56368DB680BB17648984778
:1025A000F2025AD4B3020CD5D4F85480DFF8C8A193
:1025B00000274FF00109A36D9B68F9B28B4280F0B0
:1025C0008780F70619D5616D0A6AC2F30A1702F00F
:1025D0000F0302F4F012B2F5802F00F0A180B2F5E3
:1025E000402F0AD104EB830301F58051DB68186AA0
:1025F00000231A469F4240F087803003D5F81848E0
:1026000013D5E10302D50020FFF7B2FEA20302D5E5
:102610000120FFF7ADFE630302D50220FFF7A8FEFD
:10262000270302D50320FFF7A3FE750384D5E00737
:1026300002D50020FFF730FFA10702D50120FFF7E8
:102640002BFF620702D50220FFF726FF23077FF545
:1026500073AF0320FFF720FF6EE7D4F85480DFF854
:1026600018A100274FF00109A36D9B685FFA87FB53
:102670005B4597D308EB4B13D3F8002902F44022B3
:10268000B2F5802F22D1D3F80029002A1EDAD3F820
:10269000002942F09042C3F80029D3F80029002A0B
:1026A000FBDB5946606DFFF73DFC228909FA0BF30D
:1026B00022EA0303238104EB8B03DB689B6813B1DD
:1026C0005946504698475846FFF736FC0137CBE746
:1026D00008EB4112D2F8003B03F44023B3F5802FFE
:1026E00010D1D2F8003B002B0CDA628909FA01F311
:1026F00022EA0303638104EB8103DB68DB680BB12F
:1027000050469847013756E79C0708BF0A68072BD1
:1027100098BF027003F101039CBF120A013069E700
:10272000023304EB830201F580515268906902681C
:10273000D0F808C04068A2EB000E00221046974275
:102740000AD104EB830463689B699A683A449A60EF
:102750005A6817445F6050E712F0030F08BF08681B
:10276000964588BF8CF8000002F1010284BF000A80
:102770000CF1010CE3E700BF24310020436D03EBB3
:102780004111D1F8003B43F40013C1F8003B7047FE
:10279000436D03EB4111D1F8003943F40013C1F844
:1027A00000397047436D03EB4111D1F8003B23F42E
:1027B0000013C1F8003B7047436D03EB4111D1F8A2
:1027C000003923F40013C1F80039704700F1604369
:1027D00000F01F02400903F5614309018000C9B2FE
:1027E00000F1604083F8001300F56140012393403D
:1027F000C0F880310360704730B5039C0172043328
:1028000004FB0325C361049B03630021059B006057
:102810004060C1604261026185610462426281621E
:10282000C162436330BD00000022416A4161016121
:10283000C2608262C2626FF00101FFF727B8000038
:1028400003694269934203D1C2680AB1002070470C
:10285000181D704703691960C2680132C260C269FD
:10286000134482690361934224BF436A03610021D8
:10287000FFF700B838B504460D46E3683BB162691E
:10288000131D1268A3621344E362002038BD237A4B
:1028900033B929462046FEF7DDFF0028EDDA38BDC2
:1028A0006FF00100FBE70000C368C269013BC36031
:1028B0004369134482694361934224BF436A43617D
:1028C00000238362036B03B11847704770B5202360
:1028D000044683F31188866A3EB9FFF7CBFF0546AD
:1028E00018B186F31188284670BDA36AE26A13F80E
:1028F000015BA362934202D32046FFF7D5FF00237A
:1029000083F31188EFE700002DE9F84F04460E46E7
:1029100090469946202787F311880025AA46D4F8C7
:1029200028B0BBF1000F09D149462046FFF7A2FFAE
:1029300020B18BF311882846BDE8F88FA16AE36ABD
:10294000A8EB050B5B1A9B4528BF9B46BBF1400FCC
:102950001BD9334601F1400251F8040B43F8040B34
:102960009142F9D1A36A40334036A3624035A26A4E
:10297000E36A9A4202D32046FFF796FF8AF3118852
:102980004545D8D287F31188C9E730465A46FEF745
:10299000B9F9A36A5B445E44A3625D44E7E70000C3
:1029A00010B5029C0172043303FB0421C3610023B0
:1029B0008362C362039B0363049B00604060C46046
:1029C00042610261816104624262436310BD0000A2
:1029D000026AC260426A4261026100228262C2628D
:1029E0006FF00101FEF752BF436902699A4203D1B9
:1029F000C2680AB100207047184650F8043B0B60CB
:102A000070470000C368C2690133C360436913445F
:102A100082694361934224BF436A43610021FEF708
:102A200029BF000038B504460D46E3683BB1236971
:102A30001A1DA262E2691344E362002038BD237AC2
:102A400033B929462046FEF705FF0028EDDA38BDE8
:102A50006FF00100FBE7000003691960C268013AEA
:102A6000C260C269134482690361934224BF436A0E
:102A7000036100238362036B03B1184770470000B2
:102A800070B5202304460E4683F31188856A35B954
:102A90001146FFF7C7FF10B185F3118870BDA36A17
:102AA0001E70A36AE26A01339342A36204D3E16910
:102AB00020460439FFF7D0FF002080F3118870BD55
:102AC0002DE9F84F04460D4691469A464FF02008EE
:102AD00088F311880026B346A76A4FB951462046AD
:102AE000FFF7A0FF20B187F311883046BDE8F88FCB
:102AF000A06AE76AA9EB06033F1A9F4228BF1F4658
:102B0000402F1BD905F1400355F8042B40F8042B46
:102B10009D42F9D1A36A4033A3624036A26AE36AB8
:102B20009A4204D3E16920460439FFF795FF8BF3FD
:102B300011884E45D9D288F31188CDE729463A4607
:102B4000FEF7E0F8A36A3B443D44A3623E44E5E758
:102B5000026943699A4203D1C3681BB9184670479A
:102B60000023FBE7836A002BF8D0043B9B1AF5D0C7
:102B70001360C368013BC360C3691A44836902617F
:102B80009A4224BF436A0361002383620123E5E77D
:102B900000F072B9034B002258631A610222DA6016
:102BA000704700BF000C0040014B0022DA60704704
:102BB000000C0040014B5863704700BF000C004000
:102BC000FEE7000010B5174CFEF74AFDFEF76CFE5D
:102BD000802215492046FEF7F1FD012344F8180C28
:102BE0000374124B124AD96821F4E0610904090CFC
:102BF0000A431049DA60CA6842F08072CA600E491E
:102C00000A6842F001020A601022DA77202283F873
:102C10002220002383F3118862B60848BDE81040E3
:102C2000FEF7EEBDB02900208834000800ED00E07A
:102C30000003FA05F0ED00E0001000E09034000819
:102C40002DE9F84F1F4CDFF88090656904F11407F7
:102C50004FF00008D9F82430266AAA689E1B9642D5
:102C60001DD34FF0200AAA68236AD5F80CB013448C
:102C700023622B68BB425F60A6EB02066361C5F866
:102C80000C8001D1FFF790FF88F311882869D8479D
:102C90008AF311886569AB689E42E4D2DAE762691B
:102CA000BA420CD0916823628E1B9660A8680228F5
:102CB0002CBF1818981CBDE8F84FFFF77BBFBDE884
:102CC000F88F00BF88290020000C0040034B596892
:102CD0005A68521A9042FBD8704700BF001000E0BB
:102CE0004B6843608B688360CB68C3600B6943614A
:102CF0004B6903628B6943620B6803607047000095
:102D000008B5224B22481A6940F2FF110A431A61A2
:102D10001A6922F4FF7222F001021A611A691A6B11
:102D20000A431A631A6D0A431A651A4A1B6D114643
:102D3000FFF7D6FF184802F11C01FFF7D1FF174833
:102D400002F13801FFF7CCFF154802F15401FFF7FB
:102D5000C7FF144802F17001FFF7C2FF124802F1E9
:102D60008C01FFF7BDFF114802F1A801FFF7B8FF82
:102D70000F4802F1C401FFF7B3FF0E4802F1E00172
:102D8000FFF7AEFFBDE8084000F0E2B800380240AF
:102D900000000240B0340008000402400008024075
:102DA000000C0240001002400014024000180240D3
:102DB000001C02400020024008B500F039FAFFF77D
:102DC00001FFFFF761F8BDE80840FEF7F5BE00001F
:102DD00070470000064A536823F001035360EFF385
:102DE0000983683383F30988002383F311887047CC
:102DF00030EF00E010B5202383F31188104B5B689F
:102E000013F4006318D0F1EE103AEFF309844FF099
:102E1000807344F84C3C0B4BDB6844F8083CA4F14D
:102E2000680383F30988FEF7A9FC18B1064B44F840
:102E3000503C10BD054BFAE783F3118810BD00BF6D
:102E400000ED00E030EF00E031030008340300083B
:102E5000084B1A69920710B508D500241C6120237D
:102E600083F31188FFF7ECFE84F31188BDE810406E
:102E7000FFF7C0BF000C0040104B1A6C42F0080274
:102E80001A641A6E42F008021A660D4A1B6E9368A5
:102E900043F0080393600B4B53229A624FF0FF32CA
:102EA000DA6200229A615A63DA605A6001225A613A
:102EB00008211A603220FFF789BC00BF00380240A9
:102EC000002004E0000C00401F4B1A696FEAC25258
:102ED0006FEAD2521A611A69C2F308021A614FF0FE
:102EE000FF301A695A69586100215A6959615A6953
:102EF0001A6A62F080521A621A6A02F080521A62EA
:102F00001A6A5A6A58625A6A59625A6A1A6C42F0C4
:102F100080521A641A6E42F080521A661A6E0B4A78
:102F2000106840F480701060186F00F44070B0F5C5
:102F3000007F1EBF4FF4803018671967536823F471
:102F40000073536000F054B9003802400070004034
:102F5000304B4FF080521A642F4A4FF440411160B9
:102F60001A6842F001021A601A689207FCD59A6842
:102F700022F003029A60274B19469A6812F00C025D
:102F8000FBD1186800F0F90018609A601A6842F4E2
:102F900080321A600B689B03FCD54B6F43F0010332
:102FA0004B671C4B5A6F9007FCD51C4A5A601A6835
:102FB00042F080721A60184A53685904FCD5154BC8
:102FC0001A689201FCD5164A9A60164B1A68164B7D
:102FD0009A42164B1BD1164A1168164A914216D1D5
:102FE00040F205121A600B4B9A6842F002029A6096
:102FF0009A6802F00C02082AFAD15A6C42F4804214
:103000005A645A6E42F480425A665B6E704740F2D0
:103010000572E7E70038024000700040085440079E
:1030200000948838002004E011640020003C024035
:1030300000ED00E041C20F41084A08B5536911682C
:103040000B4003F00103536123B1054A13680BB130
:1030500050689847BDE80840FFF7CCBE003C0140EF
:1030600098330020084A08B5536911680B4003F0F3
:103070000203536123B1054A93680BB1D0689847A6
:10308000BDE80840FFF7B6BE003C01409833002081
:10309000084A08B5536911680B4003F004035361F3
:1030A00023B1054A13690BB150699847BDE8084040
:1030B000FFF7A0BE003C014098330020084A08B545
:1030C000536911680B4003F00803536123B1054AAB
:1030D00093690BB1D0699847BDE80840FFF78ABEF5
:1030E000003C014098330020084A08B55369116834
:1030F0000B4003F01003536123B1054A136A0BB16F
:10310000506A9847BDE80840FFF774BE003C014094
:1031100098330020174B10B55C691A68144004F40A
:1031200078725A61A30604D5134A936A0BB1D06A28
:103130009847600604D5104A136B0BB1506B984743
:10314000210604D50C4A936B0BB1D06B9847E2056E
:1031500004D5094A136C0BB1506C9847A30504D5EC
:10316000054A936C0BB1D06C9847BDE81040FFF74F
:1031700041BE00BF003C0140983300201A4B10B5FF
:103180005C691A68144004F47C425A61620504D5F3
:10319000164A136D0BB1506D9847230504D5134A99
:1031A000936D0BB1D06D9847E00404D50F4A136EB0
:1031B0000BB1506E9847A10404D50C4A936E0BB125
:1031C000D06E9847620404D5084A136F0BB1506F54
:1031D0009847230404D5054A936F0BB1D06F9847E5
:1031E000BDE81040FFF706BE003C014098330020C8
:1031F000062108B50846FFF7E9FA06210720FFF780
:10320000E5FA06210820FFF7E1FA06210920FFF779
:10321000DDFA06210A20FFF7D9FA06211720FFF769
:10322000D5FA06212820BDE80840FFF7CFBA0000F4
:1032300008B5FFF749FE00F00BF8FDF76FFFFDF74B
:1032400043FEFFF7C5FDBDE80840FFF7A1BC000045
:10325000002304491A465A50C8180833802B42608C
:10326000F9D1704798330020034611F8012B03F879
:10327000012B002AF9D1704712101213121100000D
:1032800053544D3332463F3F3F00000000000000E2
:10329000803200083F00000013040000BC32000828
:1032A0003F00000019040000C63200083F00000083
:1032B00021040000D03200083F00000053544D3379
:1032C00032463430780053544D333246343278002D
:1032D00053544D3332463434365858000000000001
:1032E000410E00082D0E0008690E0008550E00085A
:1032F000610E00084D0E0008390E0008250E00086A
:10330000C50E0008000000000100000000000000E1
:1033100002000000000000006D100008D510000839
:1033200040004000602E0020702E002002000000AF
:103330000000000003000000000000001911000858
:103340000000000010000000802E0020000000009F
:1033500001000000000000002431002001010200F3
:1033600025424F41524425002553455249414C25A1
:1033700000565255427261696E2D763531003031FA
:1033800032333435363738394142434445460000FC
:103390004C61736572204E617669676174696F6E06
:1033A0000025424F415244252D424C00591B000834
:1033B000C5190008D90F00083D1B00084300000094
:1033C000C433000809024300020100C032090400AE
:1033D0000001020201000524001001052401000182
:1033E000042402020524060001070582030800FFE9
:1033F00009040100020A0000000705010240000064
:10340000070581024000000012000000103400088F
:103410001201100102000040AC275113000201020A
:103420000301000004030904004000000040000004
:103430000040000000400000000001000000020009
:103440000000020000000200000002000000020074
:1034500000000200000002000000000061120008ED
:1034600041150008ED15000840004000843100209F
:103470008431002001000000943100208000000011
:1034800040010000030000006D61696E0000000053
:10349000A8340008A031002098330020010000006B
:1034A000C12B00080000000069646C65000000008A
:1034B0000000802A00000000AAAAAAAA00000000BA
:1034C000FFFF00000000000000A00A000000000054
:1034D00000000000AAAAAAAA00000000FFFF000046
:1034E00000000000000000000004000000000000D8
:1034F000AAAAAAAA00000000FFFF00000000000026
:10350000000000000000001000000000AAAAAAAA03
:1035100000000000FFFF00000000000000000000AD
:103520000000000000000000AAAAAAAA00000000F3
:10353000FFFF00000000000000000000000000008D
:1035400000000000AAAAAAAA00000000FFFF0000D5
:10355000000000000000000000000000000000006B
:10356000AAAAAAAA00000000FFFF000000000000B5
:103570000000000000000000000000000A00000041
:103580000000000003000000000000000000000038
:10359000000000000000000000000000000000002B
:1035A000000000000000000000000000000000001B
:1035B000FF0096000000000804000000243400080A
:1035C00000000000000000000000000000000000FB
:0835D0000000000000000000F3
:00000001FF
